:100000000C94EC010C9409020C9409020C94090262
:100010000C9409020C9409020C9409020C94090234
:100020000C9409020C9409020C9409020C94090224
:100030000C9409020C9409020C9409020C94090214
:100040000C9409020C9409020C9409020C94090204
:100050000C9409020C9409020C9409020C940902F4
:100060000C9409020C940902E904F404FF040D0540
:100070001E052705300535053E0576302E312D321B
:100080003030383038313300485454502F312E300E
:100090002034303120556E617574686F72697A65ED
:1000A000640D0A436F6E74656E742D547970653AF1
:1000B00020746578742F68746D6C0D0A0D0A3C68A5
:1000C000313E34303120556E617574686F72697AD3
:1000D00065643C2F68313E00485454502F312E3017
:1000E00020323030204F4B0D0A436F6E74656E74B2
:1000F0002D547970653A20746578742F68746D6C2E
:100100000D0A0D0A3C68313E323030204F4B3C2FF7
:1001100068313E006574686C63642076302E312D42
:100120003230303830383133003C2F63656E7465BF
:10013000723E3C68723E3C62723E76657273696FD5
:100140006E20322E372C2074757867726170686962
:1001500063732E6F72670A00223E0A3C62723E3C55
:10016000696E70757420747970653D7375626D6920
:10017000742076616C75653D2277726974652074B0
:100180006F204C4344223E3C2F666F726D3E0A0046
:1001900071223E0A3C696E7075742073697A653D00
:1001A000323020747970653D74657874206E616DAD
:1001B000653D6C313E0A3C62723E3C696E707574FE
:1001C0002073697A653D323020747970653D7465BD
:1001D0007874206E616D653D6C323E0A3C696E70CC
:1001E000757420747970653D68696464656E206E0D
:1001F000616D653D636D642076616C75653D323E71
:100200000A3C696E70757420747970653D68696424
:1002100064656E206E616D653D70772076616C75EA
:10022000653D22003C68723E3C62723E3C666F72E5
:100230006D204D4554484F443D676574206163749B
:10024000696F6E3D220026636D643D31223E537717
:1002500069746368206F6E3C2F613E3C703E0026DF
:10026000636D643D30223E537769746368206F6626
:10027000663C2F613E3C703E00713F70773D00222E
:100280003E5B726566726573682073746174757322
:100290005D3C2F613E3C2F703E0A3C703E3C61202D
:1002A000687265663D2200713F70773D00203C61B9
:1002B00020687265663D22004F4646003C666F6EC0
:1002C0007420636F6C6F723D2223303046463030AD
:1002D000223E204F4E203C2F666F6E743E003C63E2
:1002E000656E7465723E3C703E4F75747075742017
:1002F00069733A2000485454502F312E3020323048
:1003000030204F4B0D0A436F6E74656E742D547917
:1003100070653A20746578742F68746D6C0D0A0DE1
:100320000A0071223E0A70617373776F72643A201B
:100330003C696E7075742073697A653D38207479F4
:1003400070653D2270617373776F726422206E61F5
:100350006D653D227077223E3C696E707574207425
:100360007970653D7375626D69742076616C756531
:100370003D226F6B223E3C2F666F726D3E3C2F63B9
:10038000656E7465723E003C63656E7465723E3CDA
:10039000666F726D204D4554484F443D2267657429
:1003A0002220616374696F6E3D2200485454502FBF
:1003B000312E3020323030204F4B0D0A436F6E7497
:1003C000656E742D547970653A20746578742F6861
:1003D000746D6C0D0A0D0A0011241FBECFEFD4E01E
:1003E000DEBFCDBF11E0A0E0B1E0ECE4F8E102C077
:1003F00005900D92A833B107D9F714E0A8E3B1E056
:1004000001C01D92AF34B107E1F70E94C6030C94FE
:10041000240C0C940000CF93DF93EC01FB0140E02F
:1004200010C08081981759F431968081882341F457
:10043000219688818D3319F4FB0141E001C0FB0155
:1004400021969881992329F0903219F0442349F399
:1004500002C04130C1F49C2FA7E2B4E002C08D93EA
:1004600021969E01291BE22F8881882341F080324A
:1004700031F0863221F034E0AD33B30781F7F0E09C
:10048000E95DFB4F1082842FDF91CF910895982F63
:1004900080538A3068F08153863010F4865F089567
:1004A000892F8154863010F080E00895892F87537A
:1004B0000895CF93DF93DC01EC0136C08B3211F449
:1004C00080E230C0853271F5FD013196DF01119671
:1004D0009081392F30533A3070F0892F8156863011
:1004E00010F4375208C0892F8154863010F030E064
:1004F00002C0392F37532181922F90539A3070F0D8
:10050000822F8156863010F4975208C0822F815472
:10051000863010F090E002C0922F9753832F82957F
:10052000807F892B899311968C91882339F61882C4
:10053000DF91CF910895EF92FF920F931F93CF9386
:10054000DF937C018B01C0E0D0E007C0F701EC0F26
:10055000FD1F80810E94030B2196C017D107B0F3C5
:10056000CDB7DEB7E6E00C940F0C1F93CF93DF936B
:10057000EC01162F45EF52E060E070E00E94D006DB
:100580004EED52E0BC01CE010E94D006BC01112309
:1005900019F04CEB52E002C048EB52E0CE010E9451
:1005A000D006BC014DEA52E0CE010E94D0064FE1D8
:1005B00051E0BC01CE010E94E30647EA52E0BC01D3
:1005C000CE010E94D00640E351E0BC01CE010E9462
:1005D000E3064FE752E0BC01CE010E94D0064FE196
:1005E00051E0BC01CE010E94E30649E752E0BC01A4
:1005F000CE010E94D00640E351E0BC01CE010E9432
:10060000E306BC01112319F04FE552E002C046E4B5
:1006100052E0CE010E94D006BC0144E252E0CE017D
:100620000E94D0064FE151E0BC01CE010E94E306DA
:1006300040E951E0BC01CE010E94D00640E351E008
:10064000BC01CE010E94E30648E551E0BC01CE01A9
:100650000E94D00649E251E0BC01CE010E94D006C2
:10066000DF91CF911F9108950F931F938C014BEA57
:1006700053E060E070E00E94D00647E853E0BC0120
:10068000C8010E94D0064FE151E0BC01C8010E94A0
:10069000E30642E253E0BC01C8010E94D0061F916C
:1006A0000F910895EF92FF920F931F93CF93DF93D3
:1006B0007C018B01C0E0D0E007C0F701EC0FFD1F0B
:1006C00080810E94290B2196C017D107B0F3CDB7C6
:1006D000DEB7E6E00C940F0CBC0180E391E00E94D1
:1006E000D00B9C0180E0232B09F481E008951F9337
:1006F000CF93DF93EC0160E071E00E940B0288234E
:1007000011F41EEF3EC087E294E00E946C03882340
:1007100011F41FEF36C063E071E0CE010E940B02BE
:10072000882371F18091270480538A3048F5182F6F
:10073000823039F581E00E94030B67E071E0CE0161
:100740000E940B02882341F087E294E00E94590244
:1007500087E294E00E943F0B6AE071E0CE010E94C4
:100760000B02882371F061E080E00E94190B87E2A0
:1007700094E00E94590287E294E00E943F0B01C07E
:100780001DEF812FDF91CF911F910895A0E0B0E080
:10079000ECECF3E00C94EA0B80E88093610010929B
:1007A000610081E090E00E94900A52983998419A45
:1007B0003A98429A3B98439A3C98449A3D98459A75
:1007C0002198299A389A209A289885E191E00E94E8
:1007D000CD0982E00E94F1088AE090E00E94900A30
:1007E00066E774E084E10E94D40884E190E00E940E
:1007F000900A8CE00E945A0B81E00E94030B84E176
:1008000091E00E944C0B40E56BE171E085E191E0E5
:100810000E94C405BAE0BB2EA9E0AA2EF8E09F2EE4
:10082000E7E08E2EDD24D39475E0772E64E0662E0B
:1008300053E0552E42E0C42E68E371E08EEE92E064
:100840000E945609EC010097B9F3BC0188E391E0DE
:100850000E94E405882329F088E391E00E940308C0
:10086000EBCFBE0188E391E00E940006882321F3CC
:1008700080914F01813051F480915A018830E1F626
:10088000BE0188E391E00E94DB07D6CF8630A1F657
:1008900080915C0190E0009709F062C080915D0159
:1008A000803551F68091670181FF03C060E570E0FB
:1008B00065C084FFC1CF88E391E00E94A9060E9431
:1008C0009806EC01009739F48091670180FFB4CF5E
:1008D00060E570E06AC0BC01685C7E4F44E050E0B7
:1008E0008DE091E00E94D90B009719F048ED50E09F
:1008F00014C0BE01645C7E4F42E050E082E191E0B2
:100900000E94D90B009791F0CE01835C9E4F0E940C
:1009100077038F3F49F448E850E060E070E088E3F7
:1009200091E00E94D00614C08E3F29F488E391E044
:100930000E9434030DC0813011F4289A03C088232B
:1009400009F4289865B1617088E391E00E94B502CE
:10095000EC0160E570E088E391E00E941E07AEC004
:10096000099709F069CF80915D01893709F064CF5B
:100970008091670181FF07C069E779E088E391E032
:100980000E945C0759CF84FF57CF88E391E00E9413
:10099000A9068C010E9498067C01009759F4809169
:1009A000670180FF49CF69E779E088E391E00E9421
:1009B0001E0742CFEC01C85CDE4F888190E0FC014D
:1009C0003197E930F10508F05CC0EC5CFF4F0C9406
:1009D0001E0C01501040B801C701875C9E4F0E9459
:1009E0009B02D09227044FC001501040B801C701AC
:1009F000875C9E4F0E945203C092270444C05092CD
:100A0000270426B183B190E0827090709595879508
:100A10002E73282B209328042EC08981813011F455
:100A2000209A08C0823019F4209A289A04C0833092
:100A300011F4209828986092270425C08981882382
:100A400011F4409801C0409A709227041CC04AE7F4
:100A500050E060E070E088E391E00E94D0061DC0A5
:100A600080922704D092280406C0909227040E9406
:100A7000F708809328041092290407C0A092270445
:100A800002C0B09227041092280447E254E060E0CC
:100A900070E088E391E00E94E306EC0169E779E009
:100AA00088E391E00E941E0740E050E088E391E077
:100AB000E80EF91EF7018081893011F441E050E021
:100AC000BE0188E391E00E94F506B6CEEF92FF9258
:100AD0000F931F93CF93DF937C01413061F46850F3
:100AE00070409B0140E050E0685F7F4F2F5E3F4FBA
:100AF0004F4F5F4F12C0423029F020E030E040E01D
:100B000050E00BC0685070409B0140E050E0685FCF
:100B10007F4F2A5F3F4F4F4F5F4FE7018B010FC061
:100B2000F881E0E0898190E08E2B9F2BA0E0B0E07F
:100B3000280F391F4A1F5B1F2296025010400230B7
:100B4000110570F7FB01EE7FEE0DFF1D60FF0DC07C
:100B5000908180E0AA2797FDA095BA2F02C040702F
:100B60005070280F391F4A1F5B1FCA01AA27BB27D5
:100B70000097A105B10599F720953095C901CDB72A
:100B8000DEB7E6E00C940F0CAC0120E030E0F90198
:100B9000E85BFB4FDB01A20FB31F8C9180832F5FBB
:100BA0003F4F2430310599F720E030E0F901EE5B4A
:100BB000FB4FDA01A20FB31F8C9180832F5F3F4F51
:100BC0002630310599F70895FC0169327105B0F0BE
:100BD0008485883099F48585863081F4DF01969686
:100BE000E8E4F4E09C918081981741F411963196E5
:100BF00084E0EC34F807B1F781E0089580E00895CF
:100C0000CF93DF93FC016A327105C8F08485883088
:100C1000B1F48585882399F48685853481F4DF01D4
:100C2000E8E4F4E0ED019E8D8081981741F411967F
:100C3000319684E0EC34F807A9F781E001C080E048
:100C4000DF91CF910895FC01A2E4B4E08681808316
:100C50008D918683319684E0A834B807B9F708955A
:100C60000F931F938C01FC01108E118E80E4848BF6
:100C7000158A868B40E064E170E0C8010E960E9400
:100C80006605F801908F818F1F910F910895AC0137
:100C9000FC01A8E4B4E0828D868F8D91828F31961D
:100CA00084E0AC34B807B9F7CA010E943006089551
:100CB0000F931F93CF93DF93FC0182A184A383A1A1
:100CC00085A312A303A3DF01999694E08C91680F8A
:100CD000711DED018C816C83222311F08C9301C076
:100CE0001C9291501197992319F0672F7727EECF17
:100CF000222349F416A217A28091370180A711A6DA
:100D00008E5F8093370112AA13AA442351F082E028
:100D100086AB84E087AB85E080AF80E881AF80E67A
:100D200001C080E586A7DF91CF911F910F910895B3
:100D300080913E0490913F04892B19F420E030E02B
:100D400006C020914004309141042E5D3F4FC901FF
:100D50000895FC01908980E0218930E0282B392B0F
:100D600086A582958F7090E0880F991F880F991F34
:100D7000909341048093400424513040281B390B48
:100D800030933F0420933E041216130624F0109271
:100D90003F0410923E0480913E0490913F040895D8
:100DA0006A5C7F4FDC01A60FB71F6653704003C01B
:100DB0008D936F5F7F4FFA014F5F5F4F8491882360
:100DC000B9F7CB010895FA016A5C7F4FDC01A60FE9
:100DD000B71F6653704004C08D936F5F7F4F31968D
:100DE00080818823C9F7CB0108950F931F93CF9378
:100DF000DF93EC018B0188E18FA7452B11F089E18E
:100E00008FA7C8018896988B898BCE010E943006E7
:100E10001AAA1BAA045E1F4F42E0B801CE014A96EF
:100E20000E9466059AAB8BABBE01C8014A960E9430
:100E3000FB08DF91CF911F910F9108950F931F939E
:100E4000CF93DF93EC018B01FC01A2E4B4E0868137
:100E500080838D918683319684E0A834B807B9F7F2
:100E600080E18FA760913E0470913F046115710588
:100E700029F421E040E061E070E002C021E040E0C0
:100E8000CE010E945806188A88E2898BCE010E9402
:100E9000470642E06CE170E0CE014A960E9466058A
:100EA0009AAB8BABBE0186E390E00E94FB08DF911A
:100EB000CF911F910F9108950F931F93CF93DF93BD
:100EC000EC018B01FC01A2E4B4E0868180838D916A
:100ED0008683319684E0A834B807B9F7188A8CE283
:100EE000898BCE010E94470682E18FA720E041E076
:100EF00061E070E0CE010E94580642E060E270E0DE
:100F0000CE014A960E9466059AAB8BABBE018AE37E
:100F100090E00E94FB08DF91CF911F910F910895FF
:100F2000A0E0B0E0E6E9F7E00C94F20BEC017B0105
:100F3000D22E132FFC01A2E4B4E0868180838D9130
:100F40008683319684E0A834B807B9F7042F4D3D65
:100F500008F00CED188A045E098BCE010E9447064A
:100F60001CA3DDA21EA204510FA3085018A619A6A7
:100F7000DE019A9620E030E007C0F701E20FF31F90
:100F800080818D932F5F3F4F2017B8F310E0005FF3
:100F90001F4F41E0B801CE014A960E94660598A70E
:100FA00089A7BE01C8014A960E94FB08CDB7DEB7EB
:100FB000E7E00C940E0C0F931F93CF93DF93EC019B
:100FC0008B01FC01A2E4B4E0868180838D9186834D
:100FD000319684E0A834B807B9F7CE010E944706DD
:100FE0001AA28CA1883F18F08DA18F5F8DA38CA1D0
:100FF000885F8CA3BE01C8010E94FB08DF91CF91DE
:101000001F910F910895CF93DF93AC01EC0122E47F
:1010100034E0FC01D901868180838D9186833196ED
:1010200084E0A834B807B9F7FA01148A82E0858B06
:101030008E8988A3F90181919F018E8B2196F4E01E
:1010400028343F07A9F7FA017C96A8E4B4E0808130
:1010500082878D91819384E0AC34B807C1F7BA01DF
:101060008AE290E00E94FB08DF91CF9108952A98D0
:10107000962F9F71982B9EBD0DB407FEFDCF1EBC11
:101080000DB407FEFDCF67FF04C01EBC0DB407FE04
:10109000FDCF2A9A8EB508952A986F71682B6EBD80
:1010A0000DB407FEFDCF4EBD0DB407FEFDCF2A9A4D
:1010B0000895AC01FB012A988AE38EBD0DB407FEAA
:1010C000FDCF9A01DF0108C01EBC0DB407FEFDCFA5
:1010D000215030408EB58D9321153105A9F7E40FCD
:1010E000F51F10822A9A08959C01FB012A988AE72D
:1010F0008EBD0DB407FEFDCF08C080818EBD0DB43E
:1011000007FEFDCF21503040319621153105A9F75A
:101110002A9A0895482F282F30E020763070809149
:101120004C0490E028173907F9F02A988FEB8EBD10
:101130000DB407FEFDCF83E08EBD0DB407FEFDCFDD
:101140002A9A2A988FE98EBD0DB407FEFDCF85E05F
:10115000359527958A95E1F72EBD0DB407FEFDCF95
:101160002A9A407640934C0408951F93182F0E94AA
:101170008A08612F80E00E9437081F9108950F931D
:101180001F93182F062F0E948A082A981F71106437
:101190001EBD0DB407FEFDCF0EBD0DB407FEFDCF85
:1011A0002A9A1F910F9108950F931F93162F072FBF
:1011B000682F84ED0E94BF08612F86ED0E94BF0852
:1011C000602F87ED0E94BF081EE303C0812F8A9520
:1011D000F1F78AEE0E94B50880FDF8CF1F910F91BC
:1011E00008958770682F85E70E94BF08089582E7F9
:1011F0000E94B50808950F931F93CF93DF93EC01DE
:101200008B016FEF82E00E94BF0869E183E00E94DA
:10121000BF08CE018150682F86E00E94BF08CE0132
:101220008150964E692F87E00E94BF082A988AE76E
:101230008EBD0DB407FEFDCF1EBC0DB407FEFDCF65
:101240002A9A2A988AE78EBD0DB407FEFDCF09C001
:10125000F80180818EBD0DB407FEFDCF21970F5F91
:101260001F4F2097A9F72A9A2A988FE98EBD0DB4AF
:1012700007FEFDCF88E08EBD0DB407FEFDCF2A9A94
:101280008CE10E94B50881FF0CC02A988FEB8EBDBF
:101290000DB407FEFDCF88E08EBD0DB407FEFDCF77
:1012A0002A9ADF91CF911F910F910895A0E0B0E0AD
:1012B000ECE5F9E00C94EF0B6C015B0189E30E9413
:1012C000B508882319F400E010E061C060914D0476
:1012D00010914E0480E00E94BF08612F81E00E94BF
:1012E000BF0860E08AE30E943708182F60E08AE3B5
:1012F0000E943708382F20E0C12FD0E0C22BD32B1B
:10130000D0934E04C0934D0460E08AE30E943708F6
:10131000E82E60E08AE30E943708F82E60E08AE356
:101320000E943708082F10E060E08AE30E94370827
:10133000382F20E0202B312B27FD03C000E010E0E8
:1013400012C00E2D10E09F2D80E0082B192BC60136
:101350000197045010408017910708F48C01B501E3
:10136000C8010E9459086C2F8CE00E94BF086D2FA5
:101370008DE00E94BF082A988EE98EBD0DB407FE4D
:10138000FDCF80E48EBD0DB407FEFDCF2A9AC801C3
:10139000CDB7DEB7EAE00C940B0CCF93DF93EC01F2
:1013A000229A2A9A84B1886284B924982B982D981D
:1013B00080E58CBD8DB581608DBD2A988FEF8EBD87
:1013C0000DB407FEFDCF8FEF8EBD0DB407FEFDCF30
:1013D0002A9A82E390E00E94900A10924E041092A2
:1013E0004D0460E088E00E94BF0860E089E00E9450
:1013F000BF0860E08CE00E94BF0860E08DE00E94C2
:10140000BF086EEF8AE00E94BF0869E18BE00E948E
:10141000BF086FEF84E00E94BF0869E185E00E9489
:10142000BF086FEF86E00E94BF086FE187E00E946F
:10143000BF0860EB88E30E94BF086FE388E20E9468
:10144000BF0860E389E20E94BF0869EF80E30E9461
:10145000BF0867EF81E30E94BF086DE080EC0E9447
:10146000BF0860E081EC0E94BF082A9882E88EBD28
:101470000DB407FEFDCF82E38EBD0DB407FEFDCF98
:101480002A9A62E186EC0E94BF086CE087EC0E9419
:10149000BF0862E184EC0E94BF086CED8AEC0E94F8
:1014A000BF0865E08BEC0E94BF08688184EE0E9453
:1014B000BF08698185EE0E94BF086A8182EE0E94A2
:1014C000BF086B8183EE0E94BF086C8180EE0E9492
:1014D000BF086D8181EE0E94BF0860E071E080E18D
:1014E0000E94D4088FE10E948A082A988BE98EBD59
:1014F0000DB407FEFDCF80EC8EBD0DB407FEFDCF11
:101500002A9A2A988FE98EBD0DB407FEFDCF84E09C
:101510008EBD0DB407FEFDCF2A9ADF91CF910895BD
:1015200028EB3BE004C0F9013197F1F701970097F0
:10153000D1F708952FE088E190E00FB6F894A895D0
:10154000809360000FBE209360000895A8950895D1
:1015500020E33CE004C0F9013197F1F701970097CF
:10156000D1F7089587FF02C0589A01C0589886FFA6
:1015700002C0599A01C0599885FF02C05B9A01C008
:101580005B9884FF02C05C9A08955C9808950F935D
:101590001F93182F062F509A519A539A549A0E94CB
:1015A000B20A002311F05E9A01C05E985D9A81E153
:1015B0008A95F1F75D9884E08A95F1F7812F13FF02
:1015C00002C0589A01C0589882FF02C0599A01C0BF
:1015D000599881FF02C05B9A01C05B9880FF02C0EE
:1015E0005C9A01C05C98002311F05E9A01C05E987D
:1015F0005D9A81E18A95F1F75D9884E08A95F1F72B
:101600001F910F9108951F9317E2912F9A95F1F76B
:1016100060E00E94C70A1A95F1F780E39CE0FC01A4
:101620003197F1F7FC013197F1F70197F1F71F912D
:101630000895662311F4805809C0613011F4805474
:1016400005C0623011F48C5601C08C520E94030B0D
:1016500008951F9317E2912F9A95F1F761E00E9488
:10166000C70A1A95F1F780E39CE0FC013197F1F786
:10167000FC013197F1F70197F1F71F910895CF938E
:10168000DF93EC0103C00E94290B219688818823F7
:10169000D1F7DF91CF910895CF93DF93EC0102C092
:1016A0000E94290BFE01219684918823C9F7DF91BE
:1016B000CF910895FF920F931F93CF93DF93F82E4E
:1016C000509A519A539A549A569A559A2CE030E06F
:1016D00040E35CE0C0E3DCE0CA010197F1F7215090
:1016E0003040C1F780E30E94B20A5D9A01E1802F89
:1016F0008A95F1F75D9814E0812F8A95F1F7CE0174
:101700000197F1F7CE010197F1F780E30E94B20A49
:101710005D9A802F8A95F1F75D98812F8A95F1F770
:10172000CE010197F1F7CE010197F1F780E30E9416
:10173000B20A5D9A802F8A95F1F75D98812F8A957C
:10174000F1F7CE010197F1F7CE010197F1F780E2B1
:101750000E94B20A5D9A0A95F1F75D981A95F1F721
:1017600088E20E94030B88E00E94030B81E00E9444
:10177000030B86E00E94030B8F2D0E94030B87E270
:101780008A95F1F7CE010197F1F7CE010197F1F7B4
:10179000CE010197F1F7CDB7DEB7E5E00C94100C60
:1017A000FB01DC018D91019080190110D9F3990B97
:1017B0000895FB01DC014150504030F08D910190C3
:1017C000801919F40020B9F7881B990B08952F92FE
:1017D0003F924F925F926F927F928F929F92AF92C1
:1017E000BF92CF92DF92EF92FF920F931F93CF930E
:1017F000DF93CDB7DEB7CA1BDB0B0FB6F894DEBFA5
:101800000FBECDBF09942A88398848885F846E84CA
:101810007D848C849B84AA84B984C884DF80EE8014
:10182000FD800C811B81AA81B981CE0FD11D0FB61D
:10183000F894DEBF0FBECDBFED010895EE0FFF1F80
:0C1840000590F491E02D0994F894FFCF7E
:10184C00707700636D64006C31006C320047455456
:10185C0020002F20000004255455580A0100076869
:10186C007474703A2F2F31302E312E302E372F00CA
:08187C00736563726574000AD4
:00000001FF
